:1000000000180020C1000000FD100000C110000019
:10001000C1100000C1100000C1100000C11000009C
:10002000C1100000C1100000C1100000FD10000050
:10003000FD100000C11000009914000069150000B7
:10004000FD100000FD100000FD100000FD1000007C
:10005000FD100000FD100000FD100000FD1000006C
:10006000FD100000FD100000FD100000FD1000005C
:10007000351100000D120000E5120000FD10000017
:10008000FD100000FD100000FD100000FD1000003C
:10009000FD100000FD100000FD100000FD1000002C
:1000A000FD070000FD100000FD100000FD10000025
:1000B000FD100000FD100000FD100000FD1000000C
:1000C000F8B501F01FF80821474A484B1A60484A22
:1000D000484B1A60484A494B1A60494B1A780A4201
:1000E00002D01A780A431A702A22464B46481A70E0
:1000F00000234649464C1A188A4203D2E558043375
:100100001560F8E70021434B434A934201D202C3F2
:10011000FBE70023414A424958589446985004331B
:10012000C02BF9D100210326FF2580248A083D4BEE
:100130009200D2180B002F003340DB009F40106864
:100140000131B84307002000984003003B4313608F
:100150002029EBD16246344B1A608A22334B1A7045
:10016000334B663A5A707C321A709E3A9979114232
:10017000FCD0102299791142FCD10C209A792C499B
:100180000240082AFAD1053A0A713D324A71203AF2
:1001900099791142FCD0402299791142FCD0C021BA
:1001A000244A890511602021214A117014399A7955
:1001B0000A400C2AFBD1204A204B1A60204A214BCE
:1001C0001A600022204B1A60204B07321A60204A26
:1001D000204B1A6062B600F0F7F901F0B9FA00F0AE
:1001E00097FF00F0CDFEFEE7300004F034800440BD
:1001F000823F0000388004400100000F3C80044032
:1002000002D0074000E0074020FDFF1F18FEFF1F3F
:100210007C19000018FEFF1FCC00002000F9FF1F12
:100220000000000000E400E008ED00E0005006409F
:100230000040064044800440C0000505048004409E
:10024000BF5D000014E000E018E000E010E000E016
:100250000000202020ED00E0FFFFFFFFFFFFFFFF79
:10026000FFFFFFFFFFFFFFFFFFFFFFFFFFFFFFFF9E
:10027000FFFFFFFFFFFFFFFFFFFFFFFFFFFFFFFF8E
:10028000FFFFFFFFFFFFFFFFFFFFFFFFFFFFFFFF7E
:10029000FFFFFFFFFFFFFFFFFFFFFFFFFFFFFFFF6E
:1002A000FFFFFFFFFFFFFFFFFFFFFFFFFFFFFFFF5E
:1002B000FFFFFFFFFFFFFFFFFFFFFFFFFFFFFFFF4E
:1002C000FFFFFFFFFFFFFFFFFFFFFFFFFFFFFFFF3E
:1002D000FFFFFFFFFFFFFFFFFFFFFFFFFFFFFFFF2E
:1002E000FFFFFFFFFFFFFFFFFFFFFFFFFFFFFFFF1E
:1002F000FFFFFFFFFFFFFFFFFFFFFFFFFFFFFFFF0E
:10030000FFFFFFFFFFFFFFFFFFFFFFFFFFFFFFFFFD
:10031000FFFFFFFFFFFFFFFFFFFFFFFFFFFFFFFFED
:10032000FFFFFFFFFFFFFFFFFFFFFFFFFFFFFFFFDD
:10033000FFFFFFFFFFFFFFFFFFFFFFFFFFFFFFFFCD
:10034000FFFFFFFFFFFFFFFFFFFFFFFFFFFFFFFFBD
:10035000FFFFFFFFFFFFFFFFFFFFFFFFFFFFFFFFAD
:10036000FFFFFFFFFFFFFFFFFFFFFFFFFFFFFFFF9D
:10037000FFFFFFFFFFFFFFFFFFFFFFFFFFFFFFFF8D
:10038000FFFFFFFFFFFFFFFFFFFFFFFFFFFFFFFF7D
:10039000FFFFFFFFFFFFFFFFFFFFFFFFFFFFFFFF6D
:1003A000FFFFFFFFFFFFFFFFFFFFFFFFFFFFFFFF5D
:1003B000FFFFFFFFFFFFFFFFFFFFFFFFFFFFFFFF4D
:1003C000FFFFFFFFFFFFFFFFFFFFFFFFFFFFFFFF3D
:1003D000FFFFFFFFFFFFFFFFFFFFFFFFFFFFFFFF2D
:1003E000FFFFFFFFFFFFFFFFFFFFFFFFFFFFFFFF1D
:1003F000FFFFFFFFFFFFFFFFFFFFFFFFFFFFFFFF0D
:10040000FFFFFFFFFFFFFFFFFFFFFFFFDEF9FFFF23
:1004100010B5064C2378002B07D1054B002B02D0DA
:10042000044800E000BF0123237010BD18FEFF1F29
:10043000000000007C190000084B10B5002B03D011
:100440000749084800E000BF07480368002B00D1B7
:1004500010BD064B002BFBD09847F9E700000000C9
:100460001CFEFF1F7C19000018FEFF1F000000008B
:1004700010B501210D2000F033F810BD10B5FA249D
:100480000121A4000D2000F00BF8200000F082F8FC
:1004900000210D2000F004F8200000F07BF810BDD2
:1004A00010B51A2818D80C2358430C4A8358101832
:1004B0001C7D027A224205D0002901D01A710BE07E
:1004C0001A7209E043681A68002902D003210A431E
:1004D00001E002218A431A6010BDC0469C1700004B
:1004E000F0B51A282FD80C2217004743164CE519EF
:1004F0006B682600012901D0042911D150433458DA
:100500003018257D027A20202A432275A22252002B
:100510001A601A68042901D1024313E0824311E0F2
:1005200038592C7A027DA24302758022002908D016
:10053000022902D10422FF3204E00022032901D162
:10054000812252001A60F0BD9C17000072B60C4B5D
:100550001A680C4B18680C4B1B6862B65B0104D51B
:10056000322393429B415B42C018084B9A1A084BB6
:100570005A43FA239B005843920D10187047C04607
:1005800018E000E034FEFF1F04ED00E0BF5D000056
:10059000ABAA020070B50400FFF7D8FF0500002CDD
:1005A0000FD0FFF7D3FF074B401B984206D9013C01
:1005B000002C06D0FA239B00ED18F2E700F0E8FCCF
:1005C000EFE770BDE703000080221E4BD20510B597
:1005D0001A608022002012061A601B4B1B4918600B
:1005E0001B4B1C4A1960282313601B4A1B4C1360C9
:1005F0001B4A13601B4A13601B4A13601B4A13609B
:10060000092222601A4C20601A4C21601A4C236087
:100610001A4C23601A4C22601A4C20601A48016060
:100620001A490B601A490B601A4B1A6000F000FD62
:100630001920FFF7AFFF00F0BFFB1420FF30FFF7DA
:10064000A9FF10BD00E100E004800340FFBF0000EF
:10065000088003400C800340148003400080034066
:100660001C800340248003402C80034034800340DE
:1006700004900340089003400C9003401490034002
:100680000090034004A0034008A003400CA00340D6
:1006900014A0034000A003400223F0B50A4A0B4E09
:1006A0001478C8272343DB00F518686008480578EC
:1006B000002D00D1403F09040F43F75001235D4056
:1006C0005C4005701470F0BDA0FEFF1F00F8FF1F16
:1006D00018FFFF1F431E10B50020032B0ED872B663
:1006E000074A99008858002807D044685B008C505E
:1006F000044904885A5A121B5A5262B610BDC046A9
:1007000090FEFF1FC4000020F8B572B60123174AFF
:10071000082594461E00164964465A1EA25C2A42C9
:100720001AD05F017C589A00002C05D1CB190830F3
:100730005860104BCB5109E03243D2005458002C82
:100740000AD18B18083058600B4B8B500B4A13782A
:10075000013B137062B608E00133052BDCD162B6B1
:100760000022064B1A7000F09DFBF8BDE018000057
:1007700000F8FF1F88004000C80040000EFFFF1F68
:10078000421E10B5032A30D8022380001843174BAD
:10079000C0001B1872B6164CA05C03280BD800F0E2
:1007A00019FF16040207052012E0083302200FE0AB
:1007B000083304200CE00F48920014580E4B002C14
:1007C00001D1115001E09858416099500CE003208C
:1007D000A0540A0008325A60C822180700D4403AD0
:1007E000098809040A431A6062B610BD00F8FF1FA9
:1007F0004CFEFF1FE4FEFF1FF4FEFF1FF7B5BA4BD0
:100800001C781D000423E4B21C421DD0B74B1B789A
:10081000002B16D0B64A1378DBB2002B05D0013B73
:10082000DBB21370002B00D100BEB24A1378DBB2EA
:10083000002B06D0013BDBB21370002B01D100F07E
:1008400083FB0422A84B1A700822224000D14AE2FE
:10085000A94BAA4F1B78DBB29C08E4001D093C1988
:10086000002D00D0D0E1226863689006000F0138A7
:100870000C2800D9C4E100F0B7FE81018101C30159
:10088000C301C301C301C301C301A001C301C3016B
:10089000C3010D001A689A4E5B689A497360002381
:1008A0000B600121984832602060984C92B2217010
:1008B000974C3B61BB610190A24218D8D020C00088
:1008C000824200D3E1E081204000824200D1BDE0BD
:1008D00006D8802A00D1A3E0822A00D1A5E0E9E071
:1008E0008C4B9A4200D1C0E0FF33FF3313E09023DA
:1008F0001B019A4213D009D8803B9A4200D0D9E01C
:100900007A4B854C1B7823700B00D9E0834B9A42BD
:1009100000D130E1824B9A4200D1CFE0CAE03C00E6
:100920003D00B278714B20341A70A03580222368C4
:10093000134203D06068083800F0B4FA0834AC42BF
:10094000F4D100242500774BE058002805D04368F7
:10095000009300F0A7FA0098F7E7724B1851724B1A
:10096000E050724BE058002805D04368009300F037
:1009700099FA0098F7E76D4B6D4A18516D4BE050AE
:100980006B00D0526C4BE85C0238032807D800F0AB
:1009900021FE02040204002200E001225A55013522
:1009A0000434042DCFD100230124644D2B70644BFB
:1009B0006449621EE3188A5C9B001A7008231A427D
:1009C00020D000F051FA6301002805D0FA18083051
:1009D00050605D4AFA5003E0F8502B7801332B70D9
:1009E00000F042FA0122A3001343DB00002805D0E7
:1009F000FA1808305060019AFA5003E0F8502B784A
:100A00009B182B7002210023A2001143C9007B50C8
:100A100003210A438A400134BB50052CC7D14EE064
:100A20003D4C2370637002234AE07F22B08802406D
:100A3000042A3FD8384C920023706370434BD2187D
:100A4000022312781A423BD0217039E07F23B2880A
:100A50001A40042A2ED87388002B2BD102203B4940
:100A600092005218117881430DE07F23B2881A401A
:100A7000042A1FD87388002B1CD10220334992000E
:100A8000521811780143117019E07288B188304B07
:100A90005C68002C0ED01888904209D15888884292
:100AA00006D1120A032A01D1237809E01B8907E045
:100AB0000C33EDE70F22254B1A705CE000231C007D
:100AC000F5889D4200D91D002E00402D00D94026FA
:100AD00020003100FFF7E0FDA419AD1B3AD12F0033
:100AE000402E3BD047E0C0468020074017FFFF1F45
:100AF000A1FEFF1F24FFFF1F9020074000F8FF1FEB
:100B000004FFFF1F38FEFF1FC800400018FFFF1F33
:100B100081060000020300000FFFFF1F21090000F3
:100B2000210A000090FEFF1F3CFEFF1FE4FEFF1F96
:100B3000C4000020F4FEFF1F4CFEFF1F0EFFFF1F2E
:100B400030C80110E018000088004000C0200740B5
:100B5000E41800004027AF4200D92F0020003900E0
:100B6000FFF79AFDE419ED1B01D1402F03D1794B1A
:100B70001C60794B1D800122784B40E0784A79490E
:100B80001068884216D1784952688A4212D11A7880
:100B9000A92A0FD15A78452A0CD19A78C22A09D1AC
:100BA000DB786B2B06D10021704BBD3A08001A7020
:100BB000FFF772FD6E4B236022E0664F3E68002E09
:100BC00013D0654B1C882500402C00D940252900F6
:100BD0003000FFF761FD641B5F4BA4B21C80002C4A
:100BE00001D1402D00D174193C60A0225C4BD20091
:100BF0001988914204D100225A709A785D4B1A707C
:100C00000122564B1A706AE008226068013D0838DC
:100C1000EDB2134037D000F045F95749A8004258CB
:100C2000564B002A1CD0566846501100585D0831BA
:100C3000616003280BD800F0CDFC020406080321F4
:100C400004E0022102E0052100E0042159550821B9
:100C5000C8230C4200D1403B1288120413433DE0EC
:100C6000585D032808D800F0B5FC3A3A0204002287
:100C700000E001225A5532E008221440621E9441DD
:100C800002345C552BE02268110C8AB202800029E4
:100C90001ED03B4943804360AB005F58394E002F64
:100CA00001D1585001E0F158486037496D00F050CB
:100CB0006B5AD2186A5200F0D7F8002802D00830D8
:100CC000606005E0314A206013780133137006E05C
:100CD00008231C4201D12E4B00E0254B2360082243
:100CE0002C4B1A708BE5012004421ED002231B49B5
:100CF000274C0B70284B294E1A70294B1C609C60A6
:100D0000284C1A61DC600D249A615E60264B1C70D1
:100D1000FF23264C2370174C2B702270244A13702B
:100D20009F22244B1A70087013E063B2002B04DA80
:100D30000D221D4B1A7080232B700222144204D006
:100D40001A490B78DBB20B702A7010231C4200D0BA
:100D50002B70F7BD38FEFF1F0CFFFF1F94200740CC
:100D600004FFFF1F2109000301000400A1FEFF1F73
:100D7000C800400098200740E4FEFF1F4CFEFF1F04
:100D800090FEFF1F3CFEFF1FC40000200EFFFF1F50
:100D90008800400080200740A0FEFF1F50FEFF1F7C
:100DA00000F8FF1FA4FEFF1FC02007408820074057
:100DB0008C2007408420074010B500F005FB00227E
:100DC00011001B4BD150981808324160882AF9D184
:100DD00080201849C0020A6802430A601A0A1649AC
:100DE000D2B20A701A0C1549D2B20A70144A1B0EFC
:100DF0001370FF23134A00201370134A1349137012
:100E0000134A137001220A701249087012490A70BD
:100E1000124A116899430B0070210B431360802222
:100E20000F4B52041A6010220E4B1A7010BDC046B0
:100E300000F8FF1F348004409C200740B02007408A
:100E4000B4200740802007408820074094200740B6
:100E500010200740002107408420074018E400E0EC
:100E600000E100E00821074070B572B60B4D2C6818
:100E7000200000F04FFC0B2802DD62B600200CE0E1
:100E800080231B06C3409C432C6062B64823584312
:100E9000034B181800230360436070BD20FDFF1F43
:100EA000C0F9FF1F10B504000E484821201A00F0B9
:100EB000A5FB0B2814D80C4B1B78002B07D00B4B31
:100EC0001B78002B03D02000FFF71EFC08E072B651
:100ED00080231B06C340064A11680B43136062B6A9
:100EE00010BDC046C0F9FF1F0EFFFF1F17FFFF1FF9
:100EF00020FDFF1F70B5124C2368002B04D0206822
:100F000042880188130010E00E4B1B78002B03D0A1
:100F10000220FFF7DFFB20602568002DEFD10CE0F9
:100F2000C618367A002E03D001339D1A8B42F7DBA8
:100F3000002D02D1FFF7B6FF2560280070BDC04626
:100F400020FFFF1F17FFFF1F10B50B4B1B78DBB2F5
:100F5000002B0FD1094C21684A883F2A03DC8818EE
:100F600003720132F9E7402301200B80FFF708FCF0
:100F70000023236010BDC04619FFFF1F1CFFFF1F89
:100F800010B5FFF775FAFFF779FA00F001F8FAE704
:100F900070B5234C2378002B40D101332370FFF729
:100FA000A9FF002801D000F0ECFA00F0B3F8002807
:100FB00001D000F0E3FA00F019F9002801D000F0A8
:100FC000DEFA00F07FF9002801D000F0D9FA002302
:100FD0002370EFF30583002B20D1EFF3108272B65C
:100FE000104D2868002803D00F4C2178002903D029
:100FF000002A13D162B611E00123237043692B60EC
:10100000002B01D0996101E008490B60002A00D152
:1010100062B60025836845779847257070BDC04645
:1010200025FFFF1FB8000020BC000020B4000020F6
:101030001B4B1C4A19781C4B082901D1002102E0E6
:101040000A2903D12E311160132206E00C2901D1A7
:10105000283100E03C21116012221A60134B1A78EB
:10106000134B002A01D0002200E001221A60114B2C
:101070001A78114B012A01D880220CE0042A01D8E9
:10108000842208E0082A01D8852204E0102A01D829
:10109000862200E087221A600122084B1A707047EE
:1010A00024FDFF1F08B003400CB0034027FFFF1FC3
:1010B00020B0034025FDFF1F24B0034026FFFF1F83
:1010C00070B580258026ED02F6000B4C23682B427C
:1010D00001D0FFF793FB2368334201D000F02AF8D8
:1010E00023681B0501D500F091F82368DB04ECD5DB
:1010F00000F0F8F8E9E7C0463480044010B5FFF787
:10110000DFFFFFFF0022014B1A607047008104409F
:101110007047FFFF054B1878054BC0B21A78D3B261
:10112000984200D24030C01A7047C046ABFFFF1F44
:1011300029FFFF1F30B5234A13799B0611D5224B97
:10114000D479187819000130E4B200233F2800DC7C
:1011500003001E480078834203D01D48C454DBB20C
:101160000B70D1781748C9B24BB2002B17DA03794C
:101170005BB2002B13DA174B174C1D782378DBB2C8
:101180009D4202D16C23C37009E001333F2B00D98B
:1011900000231248C05CDBB2C0B2D0712370402380
:1011A00019420ED0117919420BD000210C4B197045
:1011B0000C4B1B688B4202D00B49097819722C2307
:1011C000D37030BD00A00640ABFFFF1F29FFFF1FFB
:1011D0006AFFFF1FB4FFFF1FACFFFF1F2AFFFF1FA7
:1011E00028FFFF1FB0FFFF1FAAFFFF1F054B187846
:1011F000054BC0B21A78D3B2984200D24030C01A20
:101200007047C04620000020B6FFFF1F30B5234ABC
:1012100013799B0611D5224BD47918781900013027
:10122000E4B200233F2800DC03001E48007883421C
:1012300003D01D48C454DBB20B70D1781748C9B233
:101240004BB2002B17DA03795BB2002B13DA174B82
:10125000174C1D782378DBB29D4202D16C23C370FA
:1012600009E00133272B00D900231248C05CDBB210
:10127000C0B2D0712370402319420ED011791942A7
:101280000BD000210C4B19700C4B1B688B4202D009
:101290000B49097819722C23D37030BD00B0064079
:1012A00020000020B6FFFF1FDFFFFF1F28000020E7
:1012B00021000020B7FFFF1FB5FFFF1F2400002003
:1012C0001F000020054B1878054BC0B21A78D3B226
:1012D000984200D24030C01A7047C0469C0000209F
:1012E0003100002030B52C4A13799B0623D52B4BB7
:1012F000D479187819000130E4B200233F2800DCCB
:10130000030027480078834203D02648C454D8B24B
:1013100008702549086800280DD024490978C9B209
:101320008B4201D35B1A01E05B1A4033272B02DDAD
:101330001F4B1B780371D1781748C9B24BB2002BF1
:1013400017DA03795BB2002B13DA1A4B174C1D78AE
:101350002378DBB29D4202D16C23C37009E00133D4
:10136000272B00D900231448C05CDBB2C0B2D07177
:101370002370402319420ED0117919420BD000215D
:101380000E4B19700E4B1B688B4202D00D49097829
:1013900019722C23D37030BD00C006409C00002081
:1013A000310000205B0000202C0000209D00002068
:1013B0005A000020A400002032000020300000204D
:1013C000A00000209B00002030B585B072B67022CE
:1013D0004121154B1A70154A1170154A3239117096
:1013E00080221A701A7852B2002AFBDA114B186860
:1013F00062B6114B984201D80A23584301AC0A2225
:10140000210000F0BFF800230C48E15C0500002932
:1014100005D05A008218013351800A2BF5D10133CF
:101420005B002B7005B030BD000002400700024099
:1014300006000240080002407F96980000FEFF1F51
:10144000EFF3108072B643425841C0B27047002893
:1014500000D062B67047FFFF10B5FFF7F1FF0C4AEE
:101460001468002C10D063691360002B02D0002296
:101470009A6101E0074A1360FFF7E9FF00232000AB
:101480006377A3689847E8E7FFF7E1FF10BDC04620
:10149000A8000020AC00002010B5FFF7DDFF10BD54
:1014A000164930B50B68002B02D18360C36009E098
:1014B00004681A68944207D20025121B8360C56035
:1014C000D8601A60086016E002681C689968121BF0
:1014D000026000290CD00C680B00A242F4D281609B
:1014E000C968A21AC160D860C16888601A6002E049
:1014F0008160C36098600223037530BDB000002096
:1015000070B5174D2C68002C19D02368002B02D021
:10151000013B236013E0A268002A00D0D3600021C1
:1015200020692A60036821751B6822009847636858
:10153000002BE7D023602000FFF7B2FFE2E7FFF7C0
:101540007FFF0022074B1C681A60FFF780FF002C0A
:1015500005D0A5682000FFF7A3FF2C00F7E770BDBA
:10156000B0000020C000002010B5034A136801330A
:101570001360FFF7C5FF10BD34FEFF1F70477047B3
:1015800070477047F8B506000D00170000243900B9
:10159000300000F0B9F80B003733DBB2092901D86D
:1015A0003031CBB230002B55390000F027F8061E41
:1015B00001D00134EBE72B1958702B005A1B9442D1
:1015C00006DD1A78295D19702A550133013CF5E7CB
:1015D0002800F8BD02B4714649084900095C490079
:1015E0008E4402BC7047C04603B4714649084000AF
:1015F0004900095A49008E4403BC70470022430841
:101600008B4274D303098B425FD3030A8B4244D3CA
:10161000030B8B4228D3030C8B420DD3FF2209020C
:1016200012BA030C8B4202D31212090265D0030BCB
:101630008B4219D300E0090AC30B8B4201D3CB03C1
:10164000C01A5241830B8B4201D38B03C01A524103
:10165000430B8B4201D34B03C01A5241030B8B4205
:1016600001D30B03C01A5241C30A8B4201D3CB02F0
:10167000C01A5241830A8B4201D38B02C01A5241D5
:10168000430A8B4201D34B02C01A5241030A8B42D8
:1016900001D30B02C01A5241CDD2C3098B4201D3F0
:1016A000CB01C01A524183098B4201D38B01C01A6E
:1016B000524143098B4201D34B01C01A52410309E5
:1016C0008B4201D30B01C01A5241C3088B4201D394
:1016D000CB00C01A524183088B4201D38B00C01A41
:1016E000524143088B4201D34B00C01A5241411A68
:1016F00000D20146524110467047FFE701B5002075
:1017000000F006F802BDC0460029F7D076E7704722
:101710007047C0461C2101231B04984201D3000CD2
:1017200010391B0A984201D3000A08391B09984254
:1017300001D30009043902A2105C40187047C0466A
:10174000040302020101010100000000000000008A
:101750000E4B70B500251E000D4CE41AA410A542D6
:1017600004D0AB00F35898470135F8E700F0FCF8D7
:10177000084B00251E00084CE41AA410A54204D012
:10178000AB00F35898470135F8E770BD74190000B5
:10179000741900007419000078190000420000F864
:1017A00040A0044001000000420000F844A00440B2
:1017B00002000000C00000F800C00440010000006A
:1017C000000000F80490044002000000000000F84F
:1017D0000890044004000000C00000F81CC0044051
:1017E00080000000C00000F810C00440100000009D
:1017F000C00000F808C0044004000000C00000F869
:101800000CC0044008000000800000F80CB0044048
:1018100008000000800000F810B004401000000034
:10182000800000F818B0044040000000800000F87C
:101830001CB0044080000000800000F814B0044098
:1018400020000000C00000F804C0044002000000B6
:10185000800000F800B0044001000000400000F8E3
:1018600000A0044001000000400000F804A0044073
:1018700002000000400000F80CA004400800000036
:10188000400000F808A0044004000000C00000F878
:1018900014C0044020000000C00000F818C004403C
:1018A00040000000800000F804B004400200000086
:1018B000800000F808B0044004000000020100F8B5
:1018C00050D0044010000000020100F854D0044041
:1018D00020000000030100F878D004404000000020
:1018E000151915190001000026FDFF1F1200000048
:1018F0000002000050FDFF1F49000000002201000F
:1019000099FDFF1F210000000021010082FDFF1F43
:101910000900000000220000BAFDFF1F1C000000AB
:101920000021000062FDFF1F09000000000300000D
:10193000FCFDFF1F000000000103090438FDFF1F2C
:101940000000000002030904D6FDFF1F0000000094
:101950000303090400FEFF1F000000000000000058
:101960000000000000000000F8B5C046F8BC08BC4C
:081970009E4670473904000097
:04197800F8B5C046B8
:10197C00FFFFFFFF0A041201100100000040C01617
:10198C00860473020102030118035400650065000C
:10199C006E00730079006400750069006E006F00C2
:1019AC0009024900020100C03209040000020300D0
:1019BC000000092111010001221C000705830340CE
:1019CC0000010705040340000109040100020300A3
:1019DC0000000921110100012221000705810340AB
:1019EC0000010705020320000206C9FF0904A15CDF
:1019FC007508150026FF0095400975810295200990
:101A0C0076910295040976B102C006ABFF0A00027A
:101A1C00A1017508150026FF00954009018102956A
:101A2C004009029102C026035400650065006E0057
:101A3C00730079006400750069006E006F0020006F
:101A4C005200610077004800490044000403090477
:101A5C000C0300000000000000000000000000006B
:081A6C00000000000000000072
:00000001FF
